:107000005FC0000078C0000076C0000074C00000BF
:1070100072C0000070C000006EC000006CC00000B4
:107020006AC0000068C0000080C4000064C00000A6
:1070300062C0000060C000005EC000005CC00000D4
:107040005AC00000BFC0000056C0000054C000007D
:1070500052C0000050C000004EC000004CC00000F4
:107060004AC0000048C0000046C0000044C0000004
:1070700042C0000040C000003EC000003CC0000014
:107080003AC0000038C0000036C0000034C0000024
:1070900032C0000030C000002EC000002CC0000034
:1070A0002AC0000028C0000026C00000FE3D173E98
:1070B000BB3E173EBB3E4C3E6E3EBB3E8E3EA03EB0
:1070C00011241FBECFEFDAE0DEBFCDBF11E0A0E09C
:1070D000B1E0E0E0FEE702C005900D92A63AB107EC
:1070E000D9F721E0A6EAB1E001C01D92A63BB207A4
:1070F000E1F716D383C684CF84E08093E9008091C2
:10710000E80085FD0EC08091E8008B778093E80051
:107110008091E80082FDF3CF8EB38111F9CF80E03A
:1071200008958091F100089593E09093E900909183
:10713000E80095FF03C08093F10008959091E80066
:107140009E779093E8009091E80090FDF4CF9EB375
:107150009111F9CF0895F89410926F001092810068
:10716000109285001092840081E085BF15BE0C94BA
:107170000000089584B7877F84BF88E10FB6F89434
:1071800080936000109260000FBE90E080E80FB620
:10719000F89480936100909361000FBE81E085BFF9
:1071A00082E085BFE1E6F0E090E8908310821092E3
:1071B00089009AEF9093880080936F0083E080931A
:1071C00081009BC31F920F920FB60F9211242F9331
:1071D0008F939F93EF93FF931092850010928400FA
:1071E000E0E0F0E085919491019649F08091A6014C
:1071F0009091A70101969093A7018093A601FF911A
:10720000EF919F918F912F910F900FBE0F901F9034
:10721000189542E061EC82E003D342E161E883E04B
:10722000FFD242E160E884E0FBC28091AE01982F7A
:107230009F77913239F59091AF01903291F0913270
:1072400009F5813AF9F48091E800877F8093E8009E
:1072500067E070E083E091E019D48091E8008B77DB
:107260000FC0813279F48091E800877F8093E80035
:1072700067E070E083E091E062D48091E8008E776F
:107280008093E80008954F925F926F927F928F9261
:107290009F92AF92BF92CF92DF92EF92FF92CF93E5
:1072A000DF9384E08093E9008091E80082FF29C2A7
:1072B00023DFD82F853481F48CE49DE19093A701DE
:1072C0008093A60107B600FCFDCFF999FECF81E1BE
:1072D00080935700E89503C0843521F40DDF8DE0DD
:1072E00023DFE6C18C34D9F38035C9F3843721F428
:1072F00084E41ADF80E0F4CF813611F489E5F0CF21
:10730000813491F4F9DEC82FF7DE90E0880F991FE1
:107310002C2F30E0322F2227330F822B932BAA27DA
:1073200097FDA095BA2F98C1803711F483E5D8CF87
:10733000833549F4CCE9D1E08991F6DE21E0C33A06
:10734000D207D1F7B5C1863521F481E3EDDE80E3C4
:10735000C7CF833731F487E8E7DE85E9E5DE8EE1E4
:10736000BFCF8536B9F4E0E0F0E083E095E08093AC
:107370005700E89507B600FCFDCF90935700E895BD
:1073800007B600FCFDCFE058FF4FE11520E7F207FC
:1073900071F7A5CF823719F4E1E0F0E00EC0863432
:1073A00019F4E0E0F0E009C08E3419F4E3E0F0E015
:1073B00004C0813539F4E2E0F0E089E080935700C1
:1073C00084918ECF823631F489E5AEDE80E0ACDE8A
:1073D00080E886CF823419F0873609F0D5C0109244
:1073E000A7011092A60188DED82E86DEE82E84DE64
:1073F000C82F8BEB8C0F823010F08FE371CFF12C04
:10740000FD2810926F00D73609F045C081E18093C6
:107410005700E8955701912CD1E0A114B10409F46B
:10742000AFC0C090A801D090A901E090AA01F0904F
:10743000AB01C634B9F4E92DF0E0EC29FD298491C3
:1074400073DE992069F082E0C80ED11CE11CF11CAA
:10745000C092A801D092A901E092AA01F092AB01DA
:107460009D2615C0D701C601B695A7959795879516
:10747000AFD45ADEE2E0CE0ED11CE11CF11CC0926A
:10748000A801D092A901E092AA01F092AB01F1E02B
:10749000AF1AB108C2CF8090A8019090A901A09026
:1074A000AA01B090AB01C63421F0C12CD12CD1E09F
:1074B00030C083E0F40180935700E89507B600FCE4
:1074C000FDCFF3CFC63461F5DD2039F14090A8013E
:1074D0005090A9016090AA017090AB010DDE2C2D97
:1074E00030E0382BF2010901D0935700E8951124C0
:1074F000F2E04F0E511C611C711C4092A801509289
:10750000A9016092AA017092AB01DD2621E0E21A86
:10751000F108E114F104B1F627C0EEDDC82EF5CF75
:10752000EBDD682F8091A8019091A901A091AA019B
:10753000B091AB01B695A7959795879551D4409199
:10754000A8015091A9016091AA017091AB014E5F11
:107550005F4F6F4F7F4F4093A8015093A9016093F5
:10756000AA017093AB01D2CFC63441F485E0F40197
:1075700080935700E89507B600FCFDCF8DE0D4DD81
:1075800082E080936F0094C0833471F4C091A801AD
:10759000D091A901B1DD90E021E0FE010C01209322
:1075A0005700E89511249BCE833601F5C090A801C1
:1075B000D090A901E090AA01F090AB019DDDF60109
:1075C000E16090E021E00C0120935700E895112440
:1075D000F2E0CF0ED11CE11CF11CC092A801D092A8
:1075E000A901E092AA01F092AB0179CE8D3661F447
:1075F000E091A801F091A90185E080935700E895FA
:1076000007B600FCFDCF6BCE823551F4E091A801A6
:10761000F091A901C591D4918D2F86DD8C2F60CE7C
:10762000843419F569DD682F8091A8019091A90132
:10763000A091AA01B091AB01B695A79597958795B2
:10764000CFD38091A8019091A901A091AA01B091F6
:10765000AB010296A11DB11D8093A8019093A901D1
:10766000A093AA01B093AB013ACE8436F1F4C09056
:10767000A801D090A901E090AA01F090AB01D70138
:10768000C601B695A79597958795A2D34DDD22E0C3
:10769000C20ED11CE11CF11CC092A801D092A9011C
:1076A000E092AA01F092AB0103C08B3109F0A5CEA4
:1076B00083E08093E9009091E8008091E8008E7764
:1076C0008093E80095FD11C08091E80080FD04C022
:1076D0008EB38111F9CF15C08091E8008E77809329
:1076E000E80003C08EB3882361F08091E80080FF3A
:1076F000F9CF84E08093E9008091E8008B77809354
:10770000E800DF91CF91FF90EF90DF90CF90BF9096
:10771000AF909F908F907F906F905F904F90089563
:1077200080910008909101081092010810920008C1
:1077300044B714BE28E10FB6F8942093600010926D
:1077400060000FBE41FD1AC040FF09C0E0E0F0E05C
:10775000259134912F3F3F4F11F0FDDC0FC043FFC7
:107760000DC020910001309101018217930731F083
:10777000E0E0F0E085919491019679F7FBDC789454
:107780001092A7011092A60180910201882361F056
:107790007ADD07D38091A6019091A70181349F41A2
:1077A00098F310920201F0CF8091E0008160809305
:1077B000E000D1DC80E090E00895292F30E0223015
:1077C000310539F02330310549F02130310561F4BC
:1077D00010C08EE390E02CE431E01EC0882371F0ED
:1077E000813089F08230A1F080E090E020E030E04C
:1077F00013C082E190E02AE831E00EC084E090E01E
:1078000028E431E009C082E290E024E231E004C0E3
:1078100088E190E02AE031E0FA0131832083089585
:107820008093E900EBEEF0E0808181608083EDEEF3
:10783000F0E010826093EC0040838091EE00881F9E
:107840008827881F08958091AE0187FD05C080912B
:10785000E80080FF0DC010C08091E80082FD04C0E8
:107860008EB38111F9CF08958091E8008B7707C01E
:107870008EB38111ECCF08958091E8008E778093CC
:10788000E80008950F931F93CF93DF9341D048D022
:10789000C8EDD0E088818F7788838881806888836D
:1078A00088818F7D888319BC1EBA1092AC0100EECE
:1078B00010E0F80180818B7F8083888181608883DC
:1078C00042E060E080E0ACDFE1EEF0E080818E7FBE
:1078D0008083E2EEF0E08081816080838081886037
:1078E0008083F80180818E7F808388818061888396
:1078F000DF91CF911F910F910895E7EDF0E0808126
:10790000816080838AE482BF81E08093AD01BACF39
:10791000E8EDF0E080818E7F80831092E200089590
:107920001092DA001092E10008951F920F920FB6A4
:107930000F9211242F933F934F935F936F937F93F5
:107940008F939F93AF93BF93EF93FF938091DA0050
:1079500080FF1BC08091D80080FF17C08091DA00A3
:107960008E7F8093DA008091D90080FF0BC080E188
:1079700089BD82E189BD09B400FEFDCF81E08EBBE7
:107980000FD203C019BC1EBA0BD28091E10080FF58
:1079900017C08091E20080FF13C08091E2008E7FCB
:1079A0008093E2008091E20080618093E200809108
:1079B000D80080628093D80019BC85E08EBBF0D1DE
:1079C0008091E10084FF2CC08091E20084FF28C0F8
:1079D00080E189BD82E189BD09B400FEFDCF8091BF
:1079E000D8008F7D8093D8008091E1008F7E8093B6
:1079F000E1008091E2008F7E8093E2008091E200BE
:107A000081608093E2008091AC01811104C080917B
:107A1000E30087FF02C084E001C081E08EBBC0D1DB
:107A20008091E10083FF21C08091E20083FF1DC0AF
:107A30008091E100877F8093E10082E08EBB10920D
:107A4000AC018091E1008E7F8093E1008091E200A3
:107A50008E7F8093E2008091E20080618093E2005B
:107A600042E060E080E0DCDE9BD1FF91EF91BF91CE
:107A7000AF919F918F917F916F915F914F913F91C6
:107A80002F910F900FBE0F901F9018952091B40169
:107A90003091B5012617370748F06115710539F4A3
:107AA0002091E8002E772093E80001C0B901FC0185
:107AB00020E061157105A1F18EB38823E1F18530D5
:107AC000E1F18091E80083FD34C08091E80082FFFD
:107AD00006C08091E80082FF26C080E00895809172
:107AE000E80080FFE6CF2091F3008091F20090E063
:107AF000922B6115710551F08830910538F4219170
:107B00002093F100615071090196F3CF21E00897AD
:107B100009F020E08091E8008E778093E800C9CFDB
:107B20002111CACFD6CF8EB3882329F0853089F6AC
:107B300004C081E0089582E0089583E0089561150E
:107B4000710529F42091E8002B772093E800611556
:107B5000710521F12EB3222351F1253051F12091ED
:107B6000E80023FD20C02091E80022FFF3CFFC01B4
:107B7000CF014091F3002091F20030E0342B232B11
:107B800009F38091F1008193CF016150710981F770
:107B9000D9CF8EB3882359F0853059F08091E80011
:107BA00080FFF7CF02C081E0089580E0089582E071
:107BB000089583E008950F931F93CF93DF9300D030
:107BC000CDB7DEB7EEEAF1E08091F100819381E07C
:107BD000E63BF807C9F729DB8091E80083FFCBC0BB
:107BE0002091AE013091AF01832F90E08A30910552
:107BF00008F0C1C0FC01EA5AF74CE4C0223809F091
:107C0000BAC08091B20187708093E9009091EB0037
:107C10001092E9008091E800877F8093E80095FB4F
:107C2000882780F98093F1001092F10082C0822FA2
:107C30008D7F09F0A0C0223009F09DC08091B00175
:107C4000811124C02091B201277009F494C02093BF
:107C5000E9008091EB0080FF19C08091EB00333088
:107C600011F4806211C080618093EB0081E090E0AC
:107C7000022E01C0880F0A94EAF78093EA0010925E
:107C8000EA008091EB0088608093EB001092E9009D
:107C90008091E800877F50C021116DC01091B00124
:107CA0001F770FB7F8948091E800877F8093E800F2
:107CB000CADD8091E80080FFFCCF8091E3008078EE
:107CC000812B8093E30080688093E300112311F0FF
:107CD00083E001C082E08EBB0FBF4DC02058223030
:107CE00008F049C0AE014F5F5F4F6091B2018091D3
:107CF000B0019091B10161DD009709F43CC0209181
:107D0000E800277F2093E800BC0189819A81BEDECC
:107D10008091E8008B778093E8002DC0203859F5DA
:107D20008091E800877F8093E8008091AC01809388
:107D3000F1008091E8008E778093E80084DD1BC01D
:107D4000211119C09091B0019230A8F48091E800FF
:107D5000877F8093E8009093AC0175DD8091AC0142
:107D6000811104C08091E30087FF02C084E001C05C
:107D700081E08EBB4EDA8091E80083FF0AC08091DB
:107D8000EB0080628093EB008091E800877F809316
:107D9000E8000F900F90DF91CF911F910F91089500
:107DA0000895CF938EB3882359F0C091E900C7702E
:107DB0001092E9008091E80083FDFDDEC093E900A8
:107DC000CF910895EE0FFF1F0590F491E02D0994D7
:107DD000F999FECF92BD81BDF89A992780B5089593
:107DE000262FF999FECF1FBA92BD81BD20BD0FB6D7
:107DF000F894FA9AF99A0FBE01960895F894FFCF75
:107E00007777010000000000000818034B006500B0
:107E1000790062006F0061007200640069006F0009
:107E20002000000022034B006500790062006F0013
:107E300061007200640069006F00200042006F0062
:107E40006F007400200000000403090409023E00D2
:107E50000201008032090400000102020100052431
:107E60000010010424020405240600010705820312
:107E70000800FF09040100020A00000007050402CF
:107E80001000010705830210000112011001020019
:107E9000000809120023010002010001434154457A
:067EA00052494E410000B2
:040000030000700089
:00000001FF
